:020000040000FA
:020000001828BE
:08000800AB00030EAC000B116C
:10001000AA0B13282908AA00A40B13282308A4005C
:100020002208A90020142C0E8300AB0E2B0E090011
:10003000000085018316FF3090002F308500950168
:10004000F3309F00833081008312FF308500A030A1
:100050008B000130AA000130A400A2001930A300D7
:100060005C2883129F011F1451209F149F1836286B
:1000700051209F149F183A281E08A5009F011F15A4
:100080001F1451209F149F1843281E08A6009F018B
:10009000A508031D4C28A50AA608031D0800A60AEA
:1000A000080064002030A7000000000000000000ED
:1000B0000000A70B5428080000006400201C5C28E6
:1000C0002010A10AA10B6B28051231202508A300DE
:1000D0000130A1005C28A10B7D28851E70287628A0
:1000E000051D782873280530A20078280A30A20060
:1000F0001930A3000230A1005C28A10B8528051649
:100100002608A3000330A1005C28A1011930A30038
:080110000130A2005C285C280C
:02400E00AC3FC5
:00000001FF
